:100000000C944B050C9492050C9492050C9492055B
:100010000C9492050C9492050C9492050C94920504
:100020000C9492050C9492050C9423280C94F528BA
:100030000C9457230C9492050C9492050C94920501
:100040000C9492050C9492050C9492050C949205D4
:100050000C9492050C94BF230C9492050C94920579
:100060000C9492050C9492050C9492050C949205B4
:100070000C9492050C9492050C9492050C949205A4
:100080000C9492050C9492050C9492050C94920594
:100090000C9492050C9492050C9492050C94920584
:1000A0000C9492050C9492050C9492050B070D0785
:1000B00018070F0711071307150717071A071C075B
:1000C0001E072907200722072407260728072B07D2
:1000D0001719171949194919A11AA11AA11AA11A10
:1000E0008919A11A221A221A911AA11AA11A9A1A66
:1000F0002F1A2F1A2F1A2F1A2F1A2F1A2F1A2F1AB8
:100100002F1A2F1A2F1A2F1A2F1A2F1A2F1A2F1AA7
:100110003E1A4C1A531A5A1A641A261B261B381BED
:10012000381B2F1B381B381B381B261B261B341B68
:10013000381B381B341B62298929812A8929812A85
:10014000D529F829812A4F2A5E2A4C6967687400EC
:100150002D2D2D2D2D007363723A2E007363723A8C
:100160002A006361703A2E006361703A2A006E754E
:100170006D3A2E006E756D3A2A00537461747300E7
:100180002D2D2D2D2D0020554E440020524742008C
:10019000204E41560020424153004C617965720067
:1001A00001535400550056425F0060006100570043
:1001B0005C005D005E00000059005A005B0000001A
:1001C000620062006300580049004A004B0001537E
:1001D0004C004D004E000000000000000000000038
:1001E0000000520000000000500051004F000000CD
:1001F000C35CCD5CC25C0100C65CC55C0000000055
:10020000C85CC75C00000000CA5CC95C000000005C
:10021000005C00000000000000047F3F1F643214F7
:10022000643214783C1E1E140A0522232526282930
:100230002A2C2D2F3032333536383A3B3D3E404262
:10024000434547494A4C4E5051535557595A5C5EA5
:100250006062646668696B6D6F71737577797B7DB9
:100260007F81838587898A8C8E90929496989A9CB8
:100270009E9FA1A3A5A7A8AAACAEAFB1B3B4B6B8D0
:10028000B9BBBCBEBFC1C2C3C5C6C7C9CACBCCCD32
:10029000CED0D1D2D2D3D4D5D6D7D7D8D9D9DADA0D
:1002A000DBDBDBDCDCDCDCDCDDDDDDDDDCDCDCDC8D
:1002B000DCDBDBDBDADAD9D9D8D7D7D6D5D4D3D2C1
:1002C000D2D1D0CECDCCCBCAC9C7C6C5C3C2C1BF9F
:1002D000BEBCBBB9B8B6B4B3B1AFAEACAAA8A7A503
:1002E000A3A19F9E9C9A98969492908E8C8A8987BF
:1002F0008583817F7D7B79777573716F6D6B69689D
:10030000666462605E5C5A5957555351504E4C4A70
:100310004947454342403E3D3B3A3836353332301B
:100320002F2D2C2A292826252322FFAA7F5540007D
:1003300000000000000000000001010101010101B6
:100340000101020202020202020203030303030389
:10035000030404040404050505050506060606064F
:1003600007070707080808080909090A0A0A0B0B02
:100370000B0C0C0C0D0D0D0E0E0E0F0F101010119E
:10038000111212131314141515161617171818191D
:10039000191A1A1B1C1C1D1D1E1F1F202121222380
:1003A0002324252526272828292A2B2C2C2D2E2FBF
:1003B00030313132333435363738393A3B3C3D3ED3
:1003C0003F404142434445464748494B4C4D4E4FC0
:1003D00050525354555758595A5C5D5E606163647E
:1003E0006567686A6B6C6E6F7172747677797A7C08
:1003F0007D7F8182848687898B8D8E90929495975C
:10040000999B9D9FA1A2A4A6A8AAACAEB0B2B4B677
:10041000B9BBBDBFC1C3C5C8CACCCED0D3D5D7DA4E
:10042000DCDEE1E3E6E8EAEDEFF2F4F7F9FCFF00E9
:10043000AE00AF00DA02818FD9F1DB40A4A62EAF67
:1004400000A0C000A1C800AED580A81FD300408D79
:100450001420000000000000003E5B4F5B3E003EA9
:100460006B4F6B3E001C3E7C3E1C00183C7E3C18D3
:10047000001C577D571C001C5E7F5E1C0000183C52
:10048000180000FFE7C3E7FF00001824180000FF72
:10049000E7DBE7FF0030483A060E002629792926D7
:1004A00000407F05050700407F05253F005A3CE7D7
:1004B0003C5A007F3E1C1C0800081C1C3E7F001498
:1004C000227F2214005F5F005F5F0006097F017FCB
:1004D00000006689956A0060606060600094A2FF19
:1004E000A2940008047E04080010207E201000085A
:1004F000082A1C0800081C2A0808001E10101010EA
:10050000000C1E0C1E0C0030383E383000060E3E2B
:100510000E060000000000000000005F0000000068
:100520000700070000147F147F1400242A7F2A127A
:100530000023130864620036495620500000080763
:10054000030000001C224100000041221C00002A80
:100550001C7F1C2A0008083E08080000807030003C
:10056000000808080808000000606000002010086B
:100570000402003E5149453E0000427F40000072A7
:1005800049494946002141494D33001814127F1052
:10059000002745454539003C4A4949310041211170
:1005A000090700364949493600464949291E0000D5
:1005B0000014000000004034000000000814224134
:1005C00000141414141400004122140800020159EC
:1005D0000906003E415D594E007C1211127C007FDD
:1005E00049494936003E41414122007F4141413E57
:1005F000007F49494941007F09090901003E414105
:100600005173007F0808087F0000417F41000020EF
:1006100040413F01007F08142241007F404040409C
:10062000007F021C027F007F0408107F003E4141D2
:10063000413E007F09090906003E4151215E007FCD
:10064000091929460026494949320003017F01035F
:10065000003F4040403F001F2040201F003F4038E7
:10066000403F00631408146300030478040300612E
:1006700059494D4300007F414141000204081020C8
:1006800000004141417F000402010204004040405B
:100690004040000003070800002054547840007FC9
:1006A0002844443800384444442800384444287FCF
:1006B0000038545454180000087E09020018A4A4FD
:1006C0009C78007F080404780000447D40000020EE
:1006D00040403D00007F102844000000417F400062
:1006E000007C04780478007C0804047800384444D2
:1006F000443800FC182424180018242418FC007C1A
:10070000080404080048545454240004043F4424BA
:10071000003C4040207C001C2040201C003C40301D
:10072000403C004428102844004C9090907C0044A9
:1007300064544C440000083641000000007700007B
:10074000000041360800000201020402003C26239A
:10075000263C00000000000000404040F0F8F8FF98
:1007600038FFF8F83FF8F8FF38FFF8F8F04040405D
:1007700000000000000080C0C0C0800000C0C08039
:1007800000000080C0C000C0C0000080C0C00000E9
:10079000000000C0C0C0C0C000C0C0000000000019
:1007A0000000000000000000000000000000000049
:1007B0000000000000000000000000000000000039
:1007C0000000000000000000000000000000000029
:1007D0000000C0F0F8FC3E1E06010000007F414111
:1007E000417F007F4141417F000080C0E07E5B4F40
:1007F0005BFEC00000C000DCD7DEDEDED7DC00C060
:1008000000000000000000000000000000000000E8
:10081000000000000000000000494949FFFFFFFF01
:10082000E0DFBFBF00BFBFDFE0FFFFFFFF49494977
:1008300000000000001F3F6060E0BF1F007F7F07D7
:100840001E381E077F7F007F7F0E1F3B71600000F8
:100850000000007F7F0C0C0C007E7E007F7E030377
:10086000007F7E03037E7E03037F7E000F3E703C8D
:10087000063C703E0F00327B49493F7E007F7E037D
:1008800003001E3F69696F260000000000000000A1
:100890000000030F1F3F3C7870600000007F414163
:1008A000417F007F4141417F00307B7F78302020B5
:1008B00030787F3B0003000F7F0F0F0F7F0F000387
:1008C0000000000000000000000000000000000028
:1008D000000000000000000000010101070F0F7F71
:1008E0000F7F0F0F7E0F0F7F0F7F0F0F070101018B
:1008F00000000000000000000000010100000000F6
:1009000000000000000000000000000000000000E7
:1009100000000000000000000000000000000000D7
:1009200000000000000000000000000000000000C7
:1009300000000000000000000000000000000000B7
:1009400000000000000000000000000000000000A7
:100950000000000000000000000000000000000097
:100960000000000000000000000000000000000087
:100970000000000000000000000000000000000077
:100980000000000000000000000000000000000067
:100990000000000403300000000E03590061006DE8
:1009A0000070006100640000001E034D00610074CF
:1009B000007400690061002000440061006C0020A8
:1009C00000420065006E0000000403090409023BB8
:1009D00000020100A0FA090400000103010100095E
:1009E00021110100012240000705810308000A09C6
:1009F0000401000103000000092111010001223B54
:100A0000000705820320000A1201100100000008FF
:100A1000EDFE606001000102030105010906A1016C
:100A20008505050719E029E71500250195087501D9
:100A300081020508190129059505750191029501A5
:100A4000750391010507190029EF1500250195F09F
:100A500075018102C005010906A101050719E029F8
:100A6000E71500250195087501810295017508813A
:100A70000105081901290595057501910295017572
:100A80000391010507190029FF150026FF009506AF
:100A900075088100C00011241FBECFEFDAE0DEBF71
:100AA000CDBF04B603FE27C08091C2049091C30459
:100AB000A091C404B091C5048730904BA740B04BBF
:100AC000D1F41092C2041092C3041092C404109284
:100AD000C50414BE84B7877F84BF0FB6F894A89569
:100AE00080916000886180936000109260000FBE6A
:100AF000E0E0F8E3099511E0A0E0B1E0E8EAFCE508
:100B000002C005900D92AC37B107D9F724E0ACE7ED
:100B1000B1E001C01D92A23CB207E1F70E944B2553
:100B20000C94522E0C94000083E00895CF9360E063
:100B30008AE991E00E947E136091390270913A0235
:100B400080913B0290913C020E94A621813059F095
:100B500030F0823061F460E08BE891E00BC060E03F
:100B600085E991E007C060E080E991E003C060E0C2
:100B700086E891E00E9490130E947716C82F60E0EB
:100B800080E891E00E947E1360E08AE791E00E9495
:100B90007E13C0FD03C08EE691E002C084E791E0C1
:100BA00060E00E947E13C1FD03C082E691E002C0B6
:100BB00088E691E060E00E947E13C2FD03C086E5F6
:100BC00091E002C08CE591E060E00E947E1380918C
:100BD0008E0221E1622F0E94B52A482F80918D025A
:100BE0000E94B52A90918C029695969596952091A3
:100BF0008B02322F369520FD02C02EE201C02AE280
:100C00001F924F931F928F931F929F931F923F9318
:100C10001F922F9384E291E09F938F931F928CE118
:100C20008F938CE791E09F938F930E94122B60E04B
:100C300080E591E00E947E1360E08AE491E00E94EA
:100C40007E138DB79EB740960FB6F8949EBF0FBE29
:100C50008DBF60E08CE791E0CF910C94621381E04E
:100C6000089581E008950C9431061F93CF93DF938C
:100C700000D000D01F92CDB7DEB749835A836B8373
:100C80002091F10189819A81211112C0662349F0D6
:100C90000E947420182F682F89819A810E941F203A
:100CA00003C00E944920182F69817A81812F04C0D6
:100CB0000E94742069817A810F900F900F900F909D
:100CC0000F90DF91CF911F910C949C08FC01408103
:100CD00051816281738184810C9435060E94F621D2
:100CE000811102C00E9470220C94160B0C94180BF8
:100CF00008950C9478060C94790608950E94141BAC
:100D00000E947D062FEF84E39CE0215080409040BC
:100D1000E1F700C000000C94E5230F931F93CF93DD
:100D2000DF938C010E946606EC01B8010E94330635
:100D3000882309F4F7C1B801CE010E944C1588231D
:100D400009F4F0C1CA3CFCE5DF0741F4F8018281F7
:100D5000882309F4E7C10E94D90EE4C1CB3C8CE59D
:100D6000D80708F012C1C33C9CE5D90761F4F8012B
:100D70008281882309F4D6C10E94F5208272E1F0B5
:100D80000E94F410CFC1C43CECE5DE07C0F0C63CC5
:100D90009CE5D90709F4CAC008F0DCC0C43CFCE5F6
:100DA000DF0709F0CBC0F8018281882309F4BAC1BA
:100DB0000E94F520827221F30E94E710B3C1C53171
:100DC000FCE5DF0708F07BC0C2308CE5D80708F4EB
:100DD00052C0F8018281882309F454C00E94F62190
:100DE000811102C00E9470220E94092290E090931B
:100DF000B4048093B304FE01E350FC45E231F105F5
:100E000030F4EA5AFF4F8091B3040C94E92A8091A0
:100E1000B304816027C0826025C0846023C08061E4
:100E200021C080621FC080641DC080681BC08460B8
:100E3000886018C08E7F16C08D7F14C08B7F12C053
:100E40008F7E10C08F7D0EC08F7B0CC08F770AC045
:100E50008B7F877F07C087FB222720F991E09227AD
:100E600090FB87F98093B3048091B3040E940D2214
:100E70000E94141B57C1C1159CE5D90751F0C13020
:100E8000DC4579F0C801DF91CF911F910F910C944F
:100E90002F06F8018281882309F444C10E947E064E
:100EA00041C1F8018281882309F43CC18091660226
:100EB000982F909590FB80F98093660233C1C631DC
:100EC000FCE5DF0739F50E94F520982FF8018281B3
:100ED0002091170130911801882379F09A7A81E0E6
:100EE00009F480E080939901911102C069E201C088
:100EF00065E3C9010E94D8220AC08091990181113D
:100F000002C069E201C065E3C9010E94E3220E94B8
:100F1000432108C1C23CDC4509F0B4CFF80182810D
:100F2000882309F4FFC00E940211FCC0F8018281ED
:100F3000882309F4F7C00E949D0EF4C0C53CDC452F
:100F400009F0A0CFF8018281882309F4EBC00E9448
:100F5000900EE8C0F8018281C83CFCE5DF0731F45F
:100F6000882309F4DFC00E94BB0EDCC0C93CDC450D
:100F700030F4882309F4D6C00E94AC0ED3C0882375
:100F800009F4D0C00E94CA0ECDC0C13DECE5DE0719
:100F900091F4F8018281882309F4C4C00E940D0DE8
:100FA0008F3028F00E940D0D843108F405CF8FE0BA
:100FB0000E94F710B7C0C23DFCE5DF0708F05AC039
:100FC000CD3C8CE5D80739F4F8018281882309F4F7
:100FD000A9C081E0EDCFCE3C9CE5D907C0F4CB3C65
:100FE000ECE5DE0741F4F8018281882309F49AC018
:100FF0000E94150D97C0CC3CDC4509F043CFF801A9
:101000008281882309F48EC00E94260D8BC0F801CE
:101010008281CF3CFCE5DF0771F4882309F482C0AC
:101020000E940D0D863028F00E940D0D883008F4C6
:10103000C3CE86E0BDCFC03DDC4570F4882309F403
:1010400071C00E940D0D823028F00E940D0D853078
:1010500008F4B2CE82E0ACCF882309F463C00E94CA
:101060000D0D893028F00E940D0D8E3008F4A4CEAD
:1010700089E09ECFC53DECE5DE0739F4F8018281B9
:10108000882309F44FC083E293CFC63DFCE5DF0718
:1010900040F5F8018281C33DFCE5DF0729F4882390
:1010A00009F440C088E184CFC43DDC4568F488235E
:1010B000C9F10E940D0D853128F00E940D0D873178
:1010C00008F47ACE85E174CF882361F10E940D0D7A
:1010D000893128F00E940D0D823208F46DCE89E12D
:1010E00067CFCD3DECE5DE0741F4F801828188232E
:1010F000C9F082E00E94EA2515C0CE3DFCE5DF077D
:1011000039F4F8018281882369F00E9470220AC0B4
:10111000CC3DDC4509F0B6CEF8018281882311F080
:1011200080E0E8CF80E0DF91CF911F910F9108958B
:1011300080E090E008950895E72FF0E095E0899F22
:10114000E00DF11D1124EE0FFF1FEE0FFF1FE60F44
:10115000F11DEE0FFF1FE056FE4F8591949108950B
:10116000880F991FFC01E85EFD4F859194910895C9
:10117000CF93DF930E949C080E94740AEC018115B2
:10118000904508F041C0C11580E4D80708F028C197
:10119000C83ED10510F5C03ED10508F0A1C1C83A3E
:1011A000D10578F4C53AD10508F0A2C0C130D10507
:1011B00009F496C108F447C1C430D10508F090C1C4
:1011C00042C1CF3BD10508F49EC0C03CD10508F414
:1011D0003AC1CE01805C9109F5C0C11590E2D907F2
:1011E00058F4C11521E0D20708F07AC1C03FD105FB
:1011F00008F429C1D06574C1C11580E3D80708F08F
:10120000E5C0CE019F70DEC0C11595E5D90708F095
:1012100043C0C11524E5D20708F0F9C0C11582E525
:10122000D80708F5C11591E5D90708F0DCC0CE0153
:1012300074E0969587957A95E1F783709C2F93706B
:1012400021E030E002C0220F331F9A95E2F73C689C
:10125000382BCF70C695C69580E2C89FE001112457
:10126000C22BD32B3DC19E01237033278C2F869533
:101270008695C115D34508F0BBC0C1E0D0E002C0DF
:10128000CC0FDD1F2A95E2F720E2829FC0011124D6
:10129000C82BD92BDC6824C1C11529E5D207A0F4DD
:1012A000C11588E5D80708F0B7C0C11596E5D9077C
:1012B00008F0C9C08C2F0E94F00A8F71C82FD0E0AF
:1012C000DC2FCC27D0620CC1C1152AE5D20708F467
:1012D000A8C0CE0190568115904208F0B4C08D2F61
:1012E0008F710E94F00ADD27D0628F71D82BF8C071
:1012F000C53AD10509F4AAC0C63AD10509F0A9C07A
:10130000C2E8D0E4EDC0C83AD10509F4A5C0C93A95
:10131000D10509F4A4C0CA3AD10509F4A3C0CB3A57
:10132000D10509F4A2C0CC3AD10509F4A1C0CB3B48
:10133000D10509F4A0C0CC3BD10509F49FC0CD3A3A
:10134000D10509F49EC0C03BD10509F49DC0CE3A39
:10135000D10509F49CC0CF3AD10509F49BC0C13B2B
:10136000D10509F49AC0C23BD10509F499C0C33B29
:10137000D10509F498C0C43BD10509F497C0C53B19
:10138000D10509F496C0C63BD10509F495C0C73B09
:10139000D10509F494C0C83BD10509F493C0C93BF9
:1013A000D10509F492C0CD3BD10509F491C0CE3BE3
:1013B000D10509F490C0CA3BD10509F48FC0C0E043
:1013C000D4E48EC00E94B008EC018AC0CE019927F7
:1013D000D3FF03C0EC01D86C83C0EC01D06C80C09B
:1013E000DF70D06A7DC0DC2FCC27C16FD06A78C097
:1013F000C1E0D0E002C0CC0FDD1F2A95E2F720E269
:10140000829FC0011124C82BD92BDA6869C0DC2F58
:10141000CC27C46FD06A64C0DC2FCC27C06FD06AE1
:101420005FC08C2F8F700E94F00A94E0D695C7950C
:101430009A95E1F7CF70D0E0DC2FCC27D06A8F707F
:10144000806EC82B4DC0C0E0D0E04AC0C1E8D0E4F7
:1014500047C0C3E8D0E444C0C2EED4E441C0C9EE02
:10146000D4E43EC0CAEED4E43BC0C5EBD4E438C0FB
:10147000C6EBD4E435C0C3EBD4E432C0C4EBD4E44F
:101480002FC0C7EBD4E42CC0CCECD4E429C0CDEC05
:10149000D4E426C0C3E8D5E423C0CAE8D5E420C01C
:1014A000C2E9D5E41DC0C4E9D5E41AC0C1E2D6E45E
:1014B00017C0C3E2D6E414C0C4E2D6E411C0C5E24A
:1014C000D6E40EC0C6E2D6E40BC0C7E2D6E408C03C
:1014D000CFE6D4E405C0C0E7D4E402C0CAE2D6E453
:1014E000CE01DF91CF9108958238910549F1B0F492
:1014F0008133910509F459C048F48932910509F402
:101500004FC08A32910509F455C00895853391057D
:1015100009F441C08933910599F00895833E9105FE
:1015200031F138F4803E910591F0823E9105A9F0A9
:101530000895863E910501F1873E910539F10895A0
:101540002091B30420FD3BC021FD39C00895809156
:10155000B30480FF34C089E341C08091B30482FFAB
:1015600030C08091B30484FD2EC083EE37C08091DB
:10157000B30482FD26C0F5CF8091B30483FF25C05C
:101580008091B30484FD1FC087EE28C08091B3040E
:1015900083FD1BC0F5CF8091B30485FD18C019C031
:1015A0008091B30485FD15C012C08091B30486FDFF
:1015B00012C013C08091B30486FD0FC00CC080EE32
:1015C0000DC082EE0BC080E009C086EE07C089E244
:1015D00005C085E303C08AE201C081E390E008957D
:1015E0009091B30492FF0DC0282F2871283019F470
:1015F000877F846006C0282F2471243011F48B7FEC
:10160000886093FF0DC0282F2871283119F4877E38
:10161000846106C0282F2471243111F48B7E8861E7
:1016200094FD877E089508950C94130B0C94140B6D
:101630000C94130BE82FF0E0E656FE4F80810895DE
:101640000895CF93DF93A9E4B1E04EE451E061E067
:1016500070E08D91E82FE295EF70F0E091A18F702E
:101660009B0101C0220F8A95EAF7822F809589237A
:1016700081A34A175B0769F7A5E4B1E049E451E0AB
:1016800061E070E08D91E82FE295EF70F0E021A12C
:101690008F70EB0102C0CC0FDD1F8A95E2F7CE01FF
:1016A0009C2F9095922391A392A1892B82A34A17F4
:1016B0005B0741F7EFE9F1E0AAE9B1E084EA91E0E4
:1016C00011921D928E179F07D9F785E00E94FA0BA1
:1016D000DF91CF910C946E065F926F927F928F9202
:1016E0009F92AF92BF92CF92DF92EF92FF920F93B1
:1016F0001F93CF93DF9369E471E0AFE9B1E024EA8F
:10170000A22E21E0B22E612C01E010E06D015C9070
:101710001C92EB018991BE01E82FE295EF70F0E099
:1017200021A18F70A80102C0440F551F8A95E2F7CE
:10173000CA01242B21A322A1942E9094292122A313
:1017400050EA5A95F1F795E4E92E91E0F92E40E040
:1017500050E0E70189907E01282D22952F7030E01E
:10176000E90128A17C9030E0D82DDF7002C03595CA
:101770002795DA95E2F720FD08C0302F042E01C02E
:10178000330F0A94EAF7232F01C020E027292C9376
:101790004F5F5F4F44305105E1F691A1992291A22C
:1017A00092A1892B82A3119681E0F6019081951177
:1017B00001C080E0682AAA16BB0609F0A7CF262D33
:1017C00045E06AE971E08FE991E00E94FB0B0E941D
:1017D0007606862DDF91CF911F910F91FF90EF90AC
:1017E000DF90CF90BF90AF909F908F907F906F9041
:1017F0005F9008950895FF920F931F93CF93DF9307
:101800008C01F62ED72FC42F222349F081E080933C
:10181000A6010E9489239093A5018093A401809141
:10182000A6018823C1F08091A4019091A5010E9496
:101830009523069780F0EF2DFD2FD8014C2F50E017
:10184000CD01801B910B841795071CF48D9181931A
:10185000F7CF1092A601DF91CF911F910F91FF90CA
:101860000895EF92FF920F931F93CF93DF93362F3C
:10187000472F282FE82FF0E0711106C0E15DFC4FE3
:101880006491762F862F7BC0072F10E056E0659F6E
:10189000C0011124CFEFD0E0BE010E94C12A5BEA53
:1018A0005603C001579F900D1124830F911D830F84
:1018B000911D982F990F890F7E01E01AF10AEE9E73
:1018C000D001EF9EB00DFE9EB00D1124489FA001E7
:1018D0001124452F55277E01E41AF50AEE9EA0013A
:1018E000EF9E500DFE9E500D11247E01E81AF10866
:1018F000E09EC001E19E900DF09E900D1124892F75
:101900009927C81BD90BCE9FC001CF9F900DDE9F9A
:10191000900D11246230710599F050F46115710534
:10192000E9F061307105B9F48B2F722F252F18C0A3
:101930006430710561F038F06630710579F00BC0E4
:10194000892F722F02C0822F752F2B2F09C0822F53
:101950007B2F292F05C0852F7B2F02C08B2F792F3E
:10196000E22FF0E0E15DFC4F6491E72FF0E0E15DF4
:10197000FC4F7491E82FF0E0E15DFC4F8491DF9122
:10198000CF911F910F91FF90EF9008950895CF93FD
:10199000DF93762FE901682F842F0E94310C698331
:1019A00078838A83DF91CF91089580918B02282FCD
:1019B000269530E02115310519F48170826005C04B
:1019C0002532310524F08170886480938B0208955C
:1019D00088E090E00C94DB2DCF92DF92EF92FF92A3
:1019E0006B017C010E94D50CB701A60188E090E054
:1019F000FF90EF90DF90CF900C94F92DEBE8F2E0A0
:101A000083E0808311828FEF8283838314826081DD
:101A10007181828193810C94EC0C80918B0280FF08
:101A200002C08695089580E0089580918F028330EA
:101A300018F48F5F80938F0260918B0270918C02FB
:101A400080918D0290918E020C94EC0C80918F020B
:101A5000882319F0815080938F0260918B027091DE
:101A60008C0280918D0290918E020C94EC0C60910E
:101A7000040170E080918B0280FF0AC08091AB016D
:101A800023E0829FC001112480579D4F0C941012B7
:101A90008091AA0190910301891780F7E82FF0E067
:101AA0009F01220F331FE20FF31FE057FD4F1182FA
:101AB000108212828F5FF0CF90918B0290FF16C040
:101AC0009091AA0120910301921770F4E92FF0E0A0
:101AD000DF01AA0FBB1FEA0FFB1FE057FD4F8183F9
:101AE000608342839F5FF0CF0C94370D0895CF93AE
:101AF000DF9300D01F92CDB7DEB790918B0290FF9D
:101B00000AC09E012F5F3F4F0E94C70C4B81698125
:101B10008A810E945C0D0F900F900F90DF91CF9102
:101B20000895CF93DF93EC01EC81F0E0E65DFD4F8B
:101B30004491EBE8F2E0628181810E94770D8C8113
:101B40008F5F8C83DF91CF910895CF93DF93EC016A
:101B5000EBE8F2E0438162818C810E94770D8C81F9
:101B60008F5F8C83DF91CF9108950F931F93CF9355
:101B7000DF9300D01F92CDB7DEB78C018091A70113
:101B800081110AC09E012F5F3F4F4FEF6FEF0E9400
:101B9000C70C8A818093A701F8018481813051F0BC
:101BA00028F0823061F44091A7010AC08091A7011A
:101BB00040E007C06091A70140E080E003C040E042
:101BC00080E060E00E945C0DF801848190E0019665
:101BD00063E070E00E94D52A84830F900F900F90ED
:101BE000DF91CF911F910F910895AF92BF92CF9245
:101BF000DF92EF92FF920F931F93CF93DF9300D06A
:101C00001F92CDB7DEB7182FF62E042FE22E90913B
:101C10008B0290FF6DC0E92FE695AE2FB0E0A25B7E
:101C2000BE4F8C918093B3019E7F923061F49E01F0
:101C30002F5F3F4F812F0E94C70C4B8169818A81A2
:101C40000E945C0D43C0823019F400918E023EC0A8
:101C5000863019F410918C0239C08930D9F389315A
:101C6000A9F5E9518E2F8170D82EE695F0E0E65D5A
:101C7000FC4FA590B490C12CBB2460910201C61604
:101C800018F52C2D30E0A29EC001A39E900DB29EAF
:101C9000900D112470E00E94C12A812FD11002C042
:101CA000860F01C0861B9091AA01290F311DA90141
:101CB000440F551F240F351F20573D4F402F6F2DC8
:101CC0000E94C70CC394D9CF0E94370D10938C0289
:101CD000F0928D0200938E02EE2051F060918B0203
:101CE00070918C0280918D0290918E020E94EC0C7A
:101CF0000F900F900F90DF91CF911F910F91FF9058
:101D0000EF90DF90CF90BF90AF900895EBE8F2E0B6
:101D10009181282F4381628188E0890F0C94F50D11
:101D200081E00C94860EEBE8F2E09181282F43814C
:101D3000628188EF890F0C94F50D81E00C94930E6D
:101D4000EBE8F2E0628121E1620F08F46FEF282FE7
:101D5000438181810C94F50D81E00C94A00EEBE899
:101D6000F2E0628121E1621B08F460E0282F4381E8
:101D700081810C94F50D81E00C94AF0EEBE8F2E05C
:101D8000438121E1420F08F44FEF282F62818181C6
:101D90000C94F50D81E00C94BE0EEBE8F2E043816B
:101DA00021E1421B08F440E0282F628181810C94DC
:101DB000F50D81E00C94CD0E20E00C94F50DFF9212
:101DC0000F931F93CF93DF93EC01F12C0FEF10E0F3
:101DD00060910201F616F0F48091AA012F2D30E0F7
:101DE000280F311DC901880F991F280F391F20574F
:101DF0003D4F70E0C8010E94D52A962F8C814091FA
:101E00008E0260918D02F99E800D11240E94C70CF4
:101E1000F394DECF0E94370D9A818C8190FF02C02F
:101E20008F5F01C081508C83DF91CF911F910F9103
:101E3000FF900895BF92CF92DF92EF92FF920F939F
:101E40001F93CF93DF93FC01828180FF02C00FEFCD
:101E500001C001E010E0809102011817E0F58091C7
:101E6000AA01C12ED12CE601C80FD11DCE01880FC9
:101E7000991FC80FD91FC057DD4F198218821A82C7
:101E800034E0E32EF12CB12C8091A9018B0D87FF5A
:101E900003C090910201890F082E000C990BC816FF
:101EA000D90691F480918E028E9DA0018F9D500DD8
:101EB000112455954795559547959E0160918D0242
:101EC00080918C020E94C70CB00EF1E0EF1AF1086D
:101ED000D9F61F5FC0CF0E94370D8091A901013054
:101EE00031F4811102C080910201815007C090E05D
:101EF00001966091020170E00E94D52A8093A901A9
:101F0000DF91CF911F910F91FF90EF90DF90CF90D5
:101F1000BF900895CF938091AA01909103018917F2
:101F200070F4E82FF0E09F01220F331FE20FF31F40
:101F3000E057FD4F1182108212828F5FF0CFC0E018
:101F400060910201C617C0F5EC2FF0E070E0CF0100
:101F50000E94D52A2091AA01820F2091A801022E69
:101F6000000C330B90E0E217F307CCF02091010155
:101F7000022E000C330B2E173F078CF09C01220F12
:101F8000331F820F931F9C0120573D4F40918E02BB
:101F900060918D0280918C020E94C70C0BC0FC01E5
:101FA000EE0FFF1F8E0F9F1FFC01E057FD4F1182A8
:101FB00010821282CF5FC4CF0E94370D20910001A2
:101FC0008091A801820F8093A80190910101920F46
:101FD0009093010119165CF4082E000C990B4091A6
:101FE000020150E041505109841795071CF02195DA
:101FF00020930001CF9108950F931F93CF93DF9308
:102000008C01FC01848195810196817099279583CB
:102010008483C0E0D5E580910201C81700F5809166
:10202000AA012C2F30E0280F311DC901880F991FFC
:10203000280F391F20573D4F4C2F4695F8018481BA
:102040009581840F911D817040918E0260918D0267
:102050008D9F802D11240E94C70CCF5FDCCFDF91B4
:10206000CF911F910F910C94370D0F931F93CF9326
:10207000DF93EC0100E010E080910201282F30E0B6
:102080000217130724F59091AA019801290F311D19
:10209000A901440F551F240F351F20573D4F86952A
:1020A00090E04C81081719071CF4442331F002C05A
:1020B000411103C040918E0201C040E060918D0249
:1020C00080918C020E94C70C0F5F1F4FD5CF0E94DA
:1020D000370D8C8190E00196817099278C83DF9178
:1020E000CF911F910F910895EBE8F2E080818E7FF0
:1020F000808360817181828193810E94EC0C1092B7
:10210000B4012FEF80E792E0215080409040E1F74A
:1021100000C000000C94370D60918B02669570E052
:102120004BE050E085E091E00E94F82A892B19F4F9
:1021300081E08093B4010E9489239093AD01809344
:10214000AC01089590918B0290FF35C09170811180
:1021500002C0926006C0853210F0986402C0880FF9
:10216000982B90938B02662351F060918B027091B3
:102170008C0280918D0290918E020E94EC0C6091F5
:102180008B02669570E04BE050E085E091E00E94A4
:10219000F82A892B19F01092B40102C00E948C1009
:1021A00081E08093AF0140918E0260918D02809119
:1021B0008C020C94DC0E0895682F90918B029695FA
:1021C00081E0890F853208F081E00C94A21081E053
:1021D0000C94DC10682F90918B0296958FEF890FED
:1021E00009F484E20C94A21081E00C94EA1061E0FE
:1021F0000C94A210EBE8F2E08081816080838695E8
:102200000C94F71080918B0280FD0C9474100C9448
:10221000FA1060E00C94A2108091B201811133C0D9
:10222000809166028160809366020E94F62181118E
:1022300004C00E9470220E94FE0C0E94E80C609371
:102240008B0270938C0280938D0290938E026E7F2E
:1022500061F40E94FE0C0E94E80C60938B02709364
:102260008C0280938D0290938E020E94D50C109266
:10227000B40180918B0280FF03C086950E940911F2
:1022800081E08093B20108950F931F93CF93DF9362
:102290008091B401882309F48CC08091B301E0914E
:1022A0008B02E695E81BE093AE01823049F4F0E042
:1022B000EA5DFD4FE491CE2FD0E001E91DE049C079
:1022C000863049F4F0E0ED5DFD4FE491CE2FD0E093
:1022D00005EA1DE03EC0893051F4E695F0E0E05E8D
:1022E000FD4FE491CE2FD0E00FED1EE032C08F30D5
:1022F00051F4E695F0E0E35EFD4FE491CE2FD0E09F
:102300000AE11FE026C0853149F4F0E0E65EFD4FAA
:10231000E491CE2FD0E00AE81FE01BC0883181F0A5
:10232000833239F4E8E1F2E0C591D49105EB1DE088
:1023300010C0843251F4C4EFD1E005E310E109C0CC
:10234000C8EED3E00CEF1FE004C0C0EDD7E006EC10
:102350001CE08091AF01882389F01092AF010E94A8
:1023600089239E0120953095820F931F9093AD0194
:102370008093AC011092B1011092B0018091AC0138
:102380009091AD010E9495238C179D0790F0E091EC
:10239000AC01F091AD01CE0FDF1FD093AD01C09322
:1023A000AC018CEA91E0F801DF91CF911F910F9180
:1023B0000994DF91CF911F910F91089521B3342F8C
:1023C0003095232331B3432B3FB7F894FC01680FBA
:1023D000791FE617F70789F0819198E041BB00006B
:1023E00000C087FF21BB880F000000C000C000C0F4
:1023F00021BB00C09A9591F7ECCF3FBF089520B361
:10240000242B20BB9B01220F331F620F731F0E94DE
:10241000DE1187EC90E00197F1F700C0000008950D
:1024200040E10C94FF11EF92FF920F931F93CF9313
:10243000DF93EC017B0164E670E088E70E9493156E
:102440008C01EC0EFD1ECE15DF0561F017FD0AC0F4
:10245000FE01849164E670E00E94EA158C012196E9
:10246000892B89F30E946E16C801DF91CF911F91CD
:102470000F91FF90EF900895EBEAF2E080E092E098
:10248000DF019C011D9221503040E1F7F093AE0432
:10249000E093AD048FEF9FEF9093E1018093E00113
:1024A00008950E9494058093DC0180FD02C080E8BD
:1024B00001C080E28093DB010E948D156DE070E029
:1024C00086E494E00E941312892B11F080E00895B5
:1024D0008091DC0163E070E081FD03C083E494E05F
:1024E00002C080E494E00E941312892B79F76DE01A
:1024F00070E083E394E00E941312892B39F70E9465
:102500003C1281E08093DF018093DE011092DD01B7
:1025100008952091DB0136E0839FC0011124629F62
:10252000800D911D1124811522E0920714F080E0A6
:1025300090E085559D4F9093AE048093AD0408952F
:102540002091AD043091AE04255A32404091DB0118
:10255000642F70E0C9010E94C12A481B463010F464
:10256000240F311D211582E0380710F020E030E003
:1025700025553D4F3093AE042093AD040895CF937D
:10258000DF938A3029F481E0DF91CF910C943113ED
:10259000C62F682F8091AD049091AE0426E0FC0117
:1025A000A5EBB1E001900D922A95E1F7613E30F084
:1025B00026E0FC0111922A95E9F70AC0F6E06F9F28
:1025C000B00111246D5A7B4F46E050E00E94EF2A83
:1025D000C11135C0C091AD04D091AE0446E050E0C9
:1025E000BE0185EB91E00E94052B892BB1F1CB5AFE
:1025F000D2409E0185E0369527958A95E1F781E0E6
:1026000090E0AC0102C0440F551F2A95E2F72091DB
:10261000E0013091E101242B352B269645E0D6953B
:10262000C7954A95E1F702C0880F991FCA95E2F74E
:10263000822B932B9093E1018093E0010EC0E091F7
:10264000AD04F091AE049F012A5F3F4F2E173F0764
:1026500009F2808180958193F9CFDF91CF910C941D
:10266000A012CF93E82F2091AD043091AE042B5AE5
:1026700032404091DB01642F70E0C9010E94C12A01
:10268000481B842FEE2359F066E00E94B52AC82F1C
:10269000C150B0F060E080E20E94BF12F9CFA90102
:1026A000480F511D4115524018F080E020E030E005
:1026B000280F311D25553D4F3093AE042093AD04B6
:1026C000CF910895FF920F931F93CF93DF93EC0167
:1026D000F62EFC0101900020E9F78F01015011094D
:1026E000C017D10728F46F2D89910E94BF12F8CF2F
:1026F000DF91CF911F910F91FF9008951F93CF937A
:10270000DF93EC01162FFE018491882329F0612FBD
:102710000E94BF122196F7CFDF91CF911F910895AC
:102720000E947E1381E00C9431130E9489239093C0
:10273000AC048093AB048091DE0181110BC062E098
:1027400070E081E394E00E941312892B19F481E078
:102750008093DE018091DE0108956F927F928F92C7
:102760009F92AF92BF92CF92DF92EF92FF920F9320
:102770001F93CF93DF932091E0013091E101211568
:10278000310509F4D4C08091DD018111D0C061E030
:1027900070E0082F10E03B01082E02C0660C771C89
:1027A0000A94E2F7A30142235323452B11F48F5FD0
:1027B000F0CF9091DC01980165E0220F331F6A95FC
:1027C000E1F790FD12C08295880F80768093120108
:1027D000220F232F221F330B319520931501815E89
:1027E000809313011092160112C045E0369527958B
:1027F0004A95E1F7220F220F220F20931201109227
:102800001501295F2093130183E08093160124E6CC
:1028100030E047E050E060E171E088E70E941A167E
:10282000892B09F084C08091DC0180FD23C0A801C0
:1028300095E0440F551F9A95E1F745555D4F04E625
:1028400010E020E230E060E488E70E944116892B26
:1028500009F06DC00E949513E301C095D095809159
:10286000E0019091E101C823D923D093E101C09305
:10287000E0015DC080E2EBEBF1E0DF011D928A95A3
:10288000E9F785E0000F111F8A95E1F7A7E7B1E0AE
:1028900043E751E0992493942D91EA018991AE0187
:1028A000B801680F711D65557D4F30E025543E4FCE
:1028B000F90197E07F01E21AF30AA92C01C0AA0CE2
:1028C000EA94EAF77B01B12CE70189917E018A2124
:1028D000892E8B18D82DD770CD2E0D2E000CDD082B
:1028E000C82F01C0CC0FDA95EAF7D194C194D10872
:1028F000D7E0CD22DD2401C08695CA94EAF78C2B5F
:10290000D0808D298083B39488E0B812DDCF9150B8
:1029100031969F3F79F6C1E0AB37BC0709F0BCCFD9
:1029200004E610E020E230E04BEB51E08CCFDF9189
:10293000CF911F910F91FF90EF90DF90CF90BF90BC
:10294000AF909F908F907F906F9008958091DE015F
:10295000882369F062E070E08FE294E00E94131235
:10296000892B19F08091DE0108951092DE0190917B
:10297000DE0181E0892708958091DF018823B9F085
:1029800060E080E00E9489120E9496050E94AD13CB
:102990008091DE01882359F08091AB049091AC04C2
:1029A0000E94952381369A4E10F00C94A614089537
:1029B0000F931F93CF93DF93C62FD42F122FFC01B9
:1029C00082818823C9F06093E4010E948923909357
:1029D000E3018093E20180E28C0F883008F057C059
:1029E000C77081E001C0880FCA95EAF7DF91CF91E7
:1029F0001F910F910C94D4188091E401681330C09A
:102A00008091E2019091E3010E949523883C910519
:102A100038F500E20D0FCD17B9F080E28C0F883049
:102A200040F4C77081E001C0880FCA95EAF70E94A0
:102A3000DB18083028F581E09D2F977001C0880FC2
:102A40009A95EAF70E94D418812F0E94C118083085
:102A5000F0F4D77081E001C0880FDA95EAF70AC078
:102A600080E28C0F883098F4C77081E001C0880F35
:102A7000CA95EAF7DF91CF911F910F910C94DB1863
:102A8000812FDF91CF911F910F910C94C118DF918D
:102A9000CF911F910F9108959C01CB01203F4CE5F0
:102AA0003407F9F078F4283DFCE53F07B9F0293DFB
:102AB0004CE5340711F1273D3C4531F526E241EE66
:102AC00061EE1EC0223FFCE53F0799F070F0233F06
:102AD0003C45D1F427E245EE66EE12C027E245EE12
:102AE0000EC026E241EE60EE0BC027E245EE64EE3A
:102AF00007C026E241EE62EE03C028E241E065EE47
:102B00000E94D81480E00895FC018281882319F086
:102B10001092E401089581E008951092B9008CE0CC
:102B20008093B8000895EF92FF920F931F93CF9375
:102B3000DF93182FEB011092BC0084EA8093BC0055
:102B40000E9489237C018091BC0087FD0EC0CF3F8D
:102B50008FEFD807C1F30E9489238E199F098C1724
:102B60009D0788F38EEF9FEF2EC08091B900887F7C
:102B7000883041F08091B900887F803119F08FEF63
:102B80009FEF21C01093BB0084E88093BC000E949B
:102B900089238C018091BC0087FD0CC0CF3F8FEF53
:102BA000D807C1F30E948923801B910B8C179D07C6
:102BB00088F3D8CF8091B900887F883111F08034B4
:102BC000F1F680E090E0DF91CF911F910F91FF909F
:102BD000EF9008950F931F93CF93DF93EB018093B2
:102BE000BB0084E88093BC000E9489238C01809103
:102BF000BC0087FD0EC0CF3F8FEFD807C1F30E9406
:102C00008923801B910B8C179D0788F38EEF9FEF14
:102C10000CC02091B900287F81E090E0283211F4A7
:102C200080E090E0919581959109DF91CF911F917E
:102C30000F910895CF92DF92EF92FF920F931F931F
:102C4000CF93DF936B018A017901B9010E9493153B
:102C5000E6010C0D1D1DC017D10761F424E9209376
:102C6000BC00DF91CF911F910F91FF90EF90DF900B
:102C7000CF90089597FDF2CFB70189910E94EA1590
:102C8000EACFCF92DF92EF92FF920F931F93CF93F1
:102C9000DF93C62F6A017901B8010E94931597FD51
:102CA00011C0B8018C2F0E94EA15E601EC0CFD1C46
:102CB000CE15DF0539F097FD05C0B80189910E9456
:102CC000EA15F6CF24E92093BC00DF91CF911F9144
:102CD0000F91FF90EF90DF90CF90089584E980935B
:102CE000BC0008959093EA018093E9010895E09172
:102CF000E901F091EA01309721F00190F081E02D97
:102D0000099480E00895E091E901F091EA0130979B
:102D100099F020912301222359F02091B30427FF39
:102D200007C0DC012C9111962C93119725E02C9370
:102D30000280F381E02D099408952091E7013091FC
:102D4000E8012817390771F09093E8018093E701B3
:102D5000E091E901F091EA01309721F00680F781D6
:102D6000E02D099408952091E5013091E60128179E
:102D7000390771F09093E6018093E501E091E90154
:102D8000F091EA01309721F00084F185E02D09945B
:102D9000089585B7806885BF85B7806885BF089529
:102DA00008950C94D0160C94D1160C94D0160C9453
:102DB000D0160E94C9160E94D5160C94D31681E035
:102DC00008950E9480230E94210B80E00E945112EE
:102DD0000E9409240E940C110C94D716AF92BF9246
:102DE000CF92DF92EF92FF920F931F93CF93DF93D7
:102DF000CDB7DEB72A970FB6F894DEBF0FBECDBFB2
:102E00000E946C0BE82E0E94DF16811111C08FEF1B
:102E100089838A831B820E9489238160782F9D8306
:102E20008C8349815A816B818D810E949E1754C089
:102E30008CEEC82E81E0D82E00E010E0A02E802F6E
:102E40000E941A0BB82EF60121916F01F82EF2267E
:102E500031F40F5F1F4F0530110581F7D8CF8091F6
:102E6000660281FD0E94200B80E090E02F2D30E073
:102E7000482FB901082E02C0759567950A94E2F7AC
:102E800060FF25C08E83AF8281E090E06C0102C0BC
:102E9000CC0CDD1C4A95E2F72B2D30E02C213D2196
:102EA000232B09F480E088870E9489238160782F92
:102EB0009A8789874E815F8168858A850E949E17DF
:102EC000F801E451FE4F80818C25808305C0019676
:102ED0008430910569F6BDCF0E94BC14E1100E94B8
:102EE00095130E9477169091EB018917B1F00E941B
:102EF00077168093EB012A960FB6F894DEBF0FBECB
:102F0000CDBFDF91CF911F910F91FF90EF90DF9098
:102F1000CF90BF90AF900C947B062A960FB6F89492
:102F2000DEBF0FBECDBFDF91CF911F910F91FF90FC
:102F3000EF90DF90CF90BF90AF900895CF93DF9345
:102F4000CDB7DEB72B970FB6F894DEBF0FBECDBF5F
:102F50004F83588769877A878B87DE01119686E0D1
:102F6000FD0111928A95E9F785E0FE0137960190FF
:102F70000D928A95E1F749815A816B817C818D811F
:102F80009E810E94E41D2B960FB6F894DEBF0FBE03
:102F9000CDBFDF91CF910895FC01808191810E9486
:102FA000B6200895882309F4BFC0682F8CEF860FE0
:102FB000813A38F480911701909118010E94D8222B
:102FC0000CC080E2860F883050F4677081E001C049
:102FD000880F6A95EAF70E94F8200C9443218BE54C
:102FE000860F833070F4653A29F0663A31F083E851
:102FF00090E005C081E890E002C082E890E00C9487
:103000009D1688E5860F873108F08EC0683A09F46E
:1030100045C0693A09F445C06A3A09F445C06B3ABB
:1030200009F445C06C3A09F445C06B3B09F445C04E
:103030006C3B09F445C06D3A09F445C0603B09F4A6
:1030400045C06E3A09F445C06F3A09F445C0613B8A
:1030500009F445C0623B09F445C0633B09F445C02F
:10306000643B09F445C0653B09F445C0663B09F47F
:1030700045C0673B09F445C0683B09F445C0693B5E
:1030800009F445C06D3B09F445C06E3B09F445C0E9
:103090006A3B09F445C080E090E044C082EE90E0D5
:1030A00041C089EE90E03EC08AEE90E03BC085EBE7
:1030B00090E038C086EB90E035C083EB90E032C002
:1030C00084EB90E02FC087EB90E02CC08CEC90E07C
:1030D00029C08DEC90E026C083E891E023C08AE807
:1030E00091E020C082E991E01DC084E991E01AC01E
:1030F00081E292E017C083E292E014C084E292E0A1
:1031000011C085E292E00EC086E292E00BC087E239
:1031100092E008C08FE690E005C080E790E002C032
:103120008AE292E00C94B3160895882349F1682F3F
:103130008CEF860F813A38F4809117019091180135
:103140000E94E3220CC080E2860F883050F4677042
:1031500081E001C0880F6A95EAF70E94FE200C9476
:1031600043218BE5860F833020F480E090E00C94BF
:103170009D16685A673120F480E090E00C94B316F5
:103180000895CF93C82F0E94D217C93349F42FEF67
:1031900083EC99E0215080409040E1F700C00000AE
:1031A0008C2FCF910C949518882321F00E94F82041
:1031B0000C9443210895882321F00E94FE200C9452
:1031C000432108958F929F92AF92BF92DF92EF9228
:1031D000FF920F931F93CF93DF937C01062FC72F8E
:1031E000FC01D581D295DF70128111110E94152149
:1031F0000E94EE20882379F0112369F080E2800F8D
:10320000883048F082E00E948D210E94EE2091E0FB
:10321000D82ED92601C0D12CBC2EB2948FE0B82272
:103220008B2D90E0FC01E859FF4F0C94E92A8C2F7C
:10323000807FCF70882311F0C295C07F112399F051
:10324000CC2309F459C180E2800F883010F00111BD
:1032500004C08C2F0E94F82003C08C2F0E940821EC
:103260000E94432149C1802F0E949518CC2309F464
:1032700068C180E2800F883010F0011104C08C2FEB
:103280000E94FE2003C08C2F0E940E210E94432129
:1032900058C18C2F807FCF70803211F0C295C07FD3
:1032A000002319F00130C9F022C0112371F0DD2391
:1032B00041F0D13031F40E9428218C2B0E94302122
:1032C00040C10E9428218C2B1DC0DD2319F0D13074
:1032D00009F437C10E9439211AC0112321F0D630D8
:1032E00008F02FC10EC0D53008F02BC110C011233B
:1032F00061F0DD2331F0F701858180FFFDC08F7023
:1033000085838C2F0E94D4181CC1D11106C18C2F2B
:10331000B2C08C2F837009F047C011111BC1202F40
:10332000229526952770220F220F602F6F70862F0F
:1033300090E0A0E0B0E04C015D01022E04C0880CDA
:10334000991CAA1CBB1C0A94D2F704FF10C08FE082
:1033500090E0A0E0B0E004C0880F991FAA1FBB1F37
:103360002A95D2F780959095A095B09503C080E0FE
:1033700090E0DC01C695C695C370BC01CD016829FB
:1033800079298A299B29C23049F058F4C13019F0B3
:103390000E94351FDFC00E94231FDCC00E94471F10
:1033A000D9C00E94211FD6C0112319F08C2F817023
:1033B00001C08695882309F4CDC0202F229526953B
:1033C0002770220F220F602F6F70862F90E0A0E0F1
:1033D000B0E04C015D01022E04C0880C991CAA1CAF
:1033E000BB1C0A94D2F704FF10C08FE090E0A0E06D
:1033F000B0E004C0880F991FAA1FBB1F2A95D2F7FF
:1034000080959095A095B09503C080E090E0DC0198
:10341000C695C695C370BC01CD01682979298A2952
:103420009B29C23049F058F4C13019F00E94FA1FAC
:1034300091C00E94E81F8EC00E940C208BC00E9489
:103440005B1F88C0802F90E0FC01E05EF109E53150
:10345000F10508F04DC0E858FF4F0C94E92A0F70B1
:103460008C2F8F71112321F00E94811F802F4ACF52
:103470000E94A21F802F0E94DB1863C0112341F01D
:10348000D53008F05EC08C2F8F710E94C71F59C0C5
:10349000D63008F056C0F7CF112339F08C2F8F713A
:1034A0000E94811F4EC01123C9F38C2F8F710E947F
:1034B000A21F47C0112329F08C2F8F710E946C1F0F
:1034C00040C00E94671F3DC0112349F0CF718C2F6F
:1034D0000E94811F63E08C2F0E94782132C081E01E
:1034E0000E948D21D23068F182E00E948D2129C096
:1034F000112331F0DD2391F2802F0E94D21721C0D9
:10350000DD2399F2093349F4FFEF23EC89E0F15010
:1035100020408040E1F700C00000802F0E949518F5
:1035200010C04C2F4F70602FC7010E9498080E9456
:10353000921E14C04C2F4F70602FC7010E949B0831
:103540000DC098E0B91631F0B91640F086EF8B0D3A
:10355000823020F40E9477160E947B06DD20E1F085
:103560000E94EA2080FD18C0F70112820E94E42028
:103570000E94811FC7010E94D81A0E94E420DF9197
:10358000CF911F910F91FF90EF90DF90BF90AF9080
:103590009F908F900C94A21FDF91CF911F910F915C
:1035A000FF90EF90DF90BF90AF909F908F90089525
:1035B0000F931F93CF93DF93EC01988189812B8127
:1035C0003C81232B31F08F3F31F481E09F3F19F490
:1035D00003C081E001C080E080FD13C0CE010E94E5
:1035E0008D06882371F0688179818A810E94C120CB
:1035F0008C010E941E200E940F1FB801CE010E9464
:10360000E218DF91CF911F910F9108950E9415212B
:103610000E9425210C94432180911701909118015B
:103620000E94EE220C94061B0E9405210C940C1B98
:10363000E92FE295EF704E2F50E0FA013297EE300D
:10364000F105B0F4E357FF4F0C94E92A803F91F065
:1036500018F4803E68F40EC0843F51F40BC0803EE5
:1036600048F0813F29F406C093FB882780F908952C
:1036700080E0089581E008950E94B6200E94181B02
:103680000895CF93DF9300D000D01F92CDB7DEB75F
:103690000F900F900F900F900F90DF91CF910895A2
:1036A000CF93DF9300D000D000D0CDB7DEB7269601
:1036B0000FB6F894DEBF0FBECDBFDF91CF91089556
:1036C0001F93CF93DF93C091F20116E08091F30135
:1036D000C81799F0D0E01C9FF0011D9FF00D112438
:1036E000EC50FE4F408151816281738184819581CC
:1036F0000E94501B2196C770E9CFDF91CF911F9197
:103700000895409124025091250260912602709103
:10371000270280912802909129020C94501BCF938C
:103720008091290282958F7009F05FC080912602F6
:10373000882309F45AC08091F201B091F30170918D
:103740002402A0912502409127025091280291E085
:103750007F3F09F090E0692FC6E08B1709F445C060
:103760004115510521F0AF3F21F020E003C021E0D9
:1037700001C0262F90E020FD35C0C89FF001C99FF1
:10378000F00D1124EC50FE4F21812A132BC0208113
:10379000271328C02281211125C0238134812417B9
:1037A000350710F421503109241B350B283C310515
:1037B000C8F4209129022F7020612093290226E06D
:1037C000289FF001299FF00D1124E750FE4F8081C2
:1037D0008F708061808384E292E00E94D81ACF913A
:1037E0000C94601B01968770B8CFCF910895AF926B
:1037F000BF92CF92DF92EF92FF920F931F93CF93DE
:10380000DF93CDB7DEB761970FB6F894DEBF0FBE7A
:10381000CDBF8C0185E0F801DE011D9601900D926F
:103820008A95E1F7D8014C9111965C911197129607
:10383000EC903091240260912502809127029091B2
:103840002802009731F06F3F31F421E03F3F19F437
:1038500003C021E001C020E0B22FB170BB2E20FDDB
:1038600060C1F801C380D480A0902602AA2009F488
:10387000EEC020912902C816D90628F0D601A81B4F
:10388000B90BCD0104C0809590958C0D9D1DFF2432
:10389000F394883C910580F0F12C207F09F09CC0C6
:1038A0007C2DD98AC88A6E2D89890E94411B84E2A9
:1038B00092E00E94D81A2DC1822F807F09F054C057
:1038C000561314C0431312C0FE2CE1100FC02F700A
:1038D0002061209329020E94811B84E292E00E94D1
:1038E000D81A80912902F80185835CC1CD2831F076
:1038F0005F3F31F481E04F3F19F403C081E001C024
:1039000080E080FD03C081E08E2502C080E090E071
:10391000F82FF170FF2E80FF1CC08091F2012091E2
:10392000F30136E0821709F41AC190E0389FF001E4
:10393000399FF00D1124EC50FE4F6181561306C0E3
:103940006081461303C06281E61203C0019687704E
:10395000E9CFFE2CEE2009F425C180912902816077
:1039600080932902F12C1EC1561309C0431307C0CE
:10397000E11005C080912902F8018583A4C04D871C
:103980005E878D859E850E943C1B882379F1EE2001
:1039900069F120912902822F82958F7090E0029721
:1039A00074F0809124029091250298878F83198664
:1039B000DB86CA862C87CE0107960E94D81A86E03D
:1039C000F801A4E2B2E001900D928A95E1F70E941D
:1039D0008F1B0E94811B0DC0561771F04D875E87AB
:1039E0008D859E850E943C1B81111AC0C8010E94D2
:1039F000D81AFF24F394D6C04313F0CFE110EECFD2
:103A000080912902F8018583C8010E94D81A86E0B6
:103A1000E4E2F2E0DF011D928A95E9F7FA2CC2C0D8
:103A2000EE2021F320912902822F82958F7090E061
:103A300002972CF280912402909125029A83898327
:103A40001B82DD82CC822E83CE010196B6CFC816B2
:103A5000D90628F0F601E81BF90BCF0104C08095C8
:103A600090958C0D9D1D883C910548F0F12C7C2D86
:103A7000D98AC88A6E2D89890E94411B4AC0FE2CB2
:103A8000EE2009F4B3CF561333C0431331C0209155
:103A9000290220FD24C0822F82958F70482F50E08C
:103AA00041155105E1F0D80115962C9315974F302B
:103AB000510549F08F5F982F9295907F822F8F70DC
:103AC000892B15968C93C8010E94D81A86E0F801BC
:103AD000A4E2B2E001900D928A95E1F73DC086E044
:103AE000F801A4E2B2E001900D928A95E1F75AC084
:103AF0004D875E878D859E850E943C1B81115FCF1F
:103B000080912902816080932902C8010E94D81AFD
:103B100049C0E4E2F2E086E0DF011D928A95E9F710
:103B20001BC0EE2009F462CF4D875E878D859E8590
:103B30000E943C1BF82E882309F458CF86E0F80138
:103B4000A4E2B2E001900D928A95E1F784E292E05E
:103B50000E94CC170E948F1B0E94811B23C04D879F
:103B60005E878D859E850E94B620292F22952F7015
:103B7000223028F49F7039F0811105C00BC0243029
:103B800028F49F7049F4805E883020F0C8010E94BC
:103B9000D81ABF2CFB2C06C0D80115969C91907F9B
:103BA00091F7F8CF8F2D61960FB6F894DEBF0FBE58
:103BB000CDBFDF91CF911F910F91FF90EF90DF90DC
:103BC000CF90BF90AF9008951F93CF93DF93CDB761
:103BD000DEB72C970FB6F894DEBF0FBECDBF4F8374
:103BE000588769877A878B879C87CE0107960E94C2
:103BF000F71B8823D1F09F8188852A853B85232B5D
:103C000031F08F3F31F481E09F3F19F403C081E030
:103C100001C080E080FD47C04F81588569857A8565
:103C20008B859C850E94501B3EC086E0FE01379626
:103C3000DE01119601900D928A95E1F7FF81E885EA
:103C40006A857B856115710531F0EF3F31F481E0C4
:103C5000FF3F19F403C081E001C080E080FD23C074
:103C60002091F30130E0C9010196877099274091B6
:103C7000F20150E084179507F1F1F983EA837D831F
:103C80006C8396E0929FD001939FB00D1124AC50AD
:103C9000BE4FFE01319601900D929A95E1F7809307
:103CA000F3010E94601B16E08091F2019091F301F4
:103CB000891771F1189FC00111248C509E4F0E94EA
:103CC000F71B882329F1E091F2011E9FF0011124D6
:103CD000EC50FE4F408151816281738184819581D6
:103CE0000E94501B8091F20190E001968770992705
:103CF0008093F201D9CF0E94141B1092F30110920D
:103D0000F201E4E2F2E086E0DF011D928A95E9F734
:103D10002C960FB6F894DEBF0FBECDBFDF91CF91CA
:103D20001F910895EF92FF920F931F93CF93DF930C
:103D30008C01892B09F46CC0F12CEE24E394E8018A
:103D40002196F8018491843740F4843008F051C002
:103D5000813081F0823019F15BC0853709F444C0AD
:103D6000A8F19CE7980F903708F052C08F770E9417
:103D7000951841C00E5F1F4FFE01849190E2980F8D
:103D8000983050F48770FE2D01C0FF0F8A95EAF736
:103D90008F2F0E94182114C00E94D2172DC00E5FD1
:103DA0001F4FFE01849190E2980F983060F4877065
:103DB000FE2D01C0FF0F8A95EAF78F2F0E941E216A
:103DC0000E94432119C00E94951816C00E5F1F4F14
:103DD000FE01C491CC2381F08FE99FE00197F1F7B8
:103DE00000C00000C150F6CF0E5F1F4FFE01F490DF
:103DF00003C00E94D2178E018F2D882309F49FCF14
:103E0000EFE9FFE03197F1F700C000008150F5CFF6
:103E1000DF91CF911F910F91FF90EF90089508953A
:103E200008950C94101F0C94111F0E94131F60938F
:103E30003D0270933E0280933F02909340020C94A7
:103E4000061B0C94151F0F931F9300913D021091B8
:103E50003E0220913F0230914002602B712B822B59
:103E6000932B1F910F910C94151F0F931F9300918B
:103E70003D0210913E0220913F02309140026023AA
:103E80007123822393231F910F910C94151F0F937D
:103E90001F9300913D0210913E0220913F0230910C
:103EA000400260277127822793271F910F910C945E
:103EB000151F0C94101F0E94591F609339027093B4
:103EC0003A0280933B0290933C020C94061B60E004
:103ED00070E0CB010C945B1F0F931F9341E050E007
:103EE00060E070E08A019B0104C0000F111F221FD7
:103EF000331F8A95D2F7C901B8011F910F910C9415
:103F00005B1F0F931F9341E050E060E070E004C03E
:103F1000440F551F661F771F8A95D2F7809139028B
:103F200090913A02A0913B02B0913C028A019B0120
:103F3000082B192B2A2B3B2BC901B8011F910F917C
:103F40000C945B1F0F931F9341E050E060E070E022
:103F500004C0440F551F661F771F8A95D2F74095FE
:103F60005095609570958091390290913A02A09198
:103F70003B02B0913C028A019B01082319232A23AA
:103F80003B23C901B8011F910F910C945B1F0F9344
:103F90001F9341E050E060E070E004C0440F551F03
:103FA000661F771F8A95D2F78091390290913A0265
:103FB000A0913B02B0913C028A019B01082719277E
:103FC0002A273B27C901B8011F910F910C945B1F51
:103FD0000F931F930091390210913A0220913B02F6
:103FE00030913C02602B712B822B932B1F910F91F0
:103FF0000C945B1F0F931F930091390210913A02AA
:1040000020913B0230913C02602371238223932351
:104010001F910F910C945B1F0F931F930091390216
:1040200010913A0220913B0230913C0260277127A7
:10403000822793271F910F910C945B1F0895990F6E
:10404000990F890FE82FE695E695E695877051E080
:1040500001C0550F8A95EAF785E0E89FF001112429
:10406000E65DFD4F20E030E070E04081CB01022EA4
:1040700002C0969587950A94E2F78170819584270E
:104080008523842781932F5F3F4F2530310569F7C2
:104090000895990F990F890F682F66956695669513
:1040A000982F977085E0689FB001112440E050E0A0
:1040B00080E0FB01E40FF51FE65DFD4F208130E05D
:1040C000092E02C0369527950A94E2F7217033270E
:1040D000042E01C0220F0A94EAF7822B4F5F5F4F34
:1040E0004530510531F70895BF92CF92DF92EF929C
:1040F000FF920F931F93CF93DF938C01C0903902EF
:10410000D0903A02E0903B02F0903C0280913D0258
:1041100090913E02A0913F02B0914002C82AD92A54
:10412000EA2AFB2ACFE1D0E0D701C6010C2E04C059
:10413000B695A795979587950A94D2F780FD04C008
:10414000219790F7B12C07C0BC2EB8018C2F0E948C
:10415000B8080197A9F38B2DDF91CF911F910F9193
:10416000FF90EF90DF90CF90BF900895CF93DF93B3
:10417000EC010E947420BE010E94B808DF91CF912B
:1041800008951F93CF93DF93EB019091F101992351
:1041900021F0CB010E94B62013C0882349F0CB0147
:1041A0000E947420182F682FCE010E941F2004C087
:1041B000CB010E944920182FBE01812F0E94B80810
:1041C000DF91CF911F91089580914102859585954A
:1041D00085950895809141028770089590914102DC
:1041E000977081E009F480E0089580916502089558
:1041F00090916502892B8093650208958095909136
:1042000065028923809365020895109265020895DE
:1042100090916402892B8093640208958095909117
:1042200064028923809364020895109264020895C1
:1042300090916302892B80936302089580959091F9
:1042400063028923809363020895109263020895A4
:1042500080914202089508950C942B210C942C21F6
:1042600090914202981721F0809342020C942E21E3
:10427000089580914202882329F01092420280E042
:104280000C942E210895E0911701F091180180916E
:1042900065028083E0911701F0911801908180916F
:1042A0006402892B8083E0911701F09118019081BD
:1042B00080916302892B808380914202882381F060
:1042C000E0911701F09118019081892B80838091F2
:1042D0001701909118010E94722281110E943921C8
:1042E00080911701909118010C9483160C942B2146
:1042F00098E0899F90011124262B209341020E946F
:10430000811F809141028595859585950C94762134
:104310001092410280E00C94762120914102809518
:10432000822380934102982F977079F430E0482FD0
:10433000082E000C550B2417350739F08595859507
:1043400085950E94A21F0C9488210895CF92DF9238
:10435000EF92FF926C01EE24FF24C114D104E1041A
:10436000F10421F0C701B60120E101C020E0C72E11
:10437000D82EE92EFF24C114D104E104F10419F070
:10438000285FC701B6016B017C0154E0F694E79405
:10439000D794C7945A95D1F7C114D104E104F1041C
:1043A00019F02C5FC701B6016B017C0142E0F69465
:1043B000E794D794C7944A95D1F7C114D104E10486
:1043C000F10419F02E5FC701B601DC01CB01B695EF
:1043D000A79597958795892B8A2B8B2B09F02F5FB3
:1043E000822FFF90EF90DF90CF90089580E090E0D3
:1043F0000E94E12D21E08D3E9E4F09F020E0822FAA
:10440000089582E090E00C94D32D83E090E00C942A
:10441000D32D84E090E00C94D32D682F84E090E0BD
:104420000C94E72DAB01BC018FE090E00C94F92DCA
:10443000AB01BC0183E190E00C94F92D60E070E0E9
:10444000CB010C94182260E070E0CB010E94122294
:104450000C941E226DEE7EEF80E090E00E94052E0F
:1044600060E082E090E00E94E72D60E083E090E071
:104470000E94E72D10923D0210923E0210923F02E0
:104480001092400260E084E090E00E94E72D60E03E
:1044900085E090E00E94E72D60E086E090E00E94D9
:1044A000E72D6FEF87E090E00E94E72D40E050E0BD
:1044B000BA0188E090E00E94F92D60E08DE090E084
:1044C0000E94E72D40E050E0BA0188E190E00E94B0
:1044D000F92D60E087E190E00E94E72D0C94232203
:1044E0000C942A22FC01329680912301882331F01A
:1044F0008091B30487FF02C09EE101C096E080E096
:10450000915028F021912223D9F38F5FF9CF08959C
:104510009C01FC0132969FEF80E04191461789F0A3
:104520009F3F19F4411101C0982F8F5F8630A9F782
:104530009F3F39F0F901E90FF11D97FDFA9562836C
:10454000089508959C012A5F3F4FFC014281461364
:1045500001C01282019682179307B9F70895262F9A
:104560002695269526952E3168F4FC01E20FF11D63
:10457000677021E030E001C0220F6A95EAF782817E
:10458000282B22830895262F2695269526952E31B1
:1045900070F4FC01E20FF11D677021E030E001C012
:1045A000220F6A95EAF720958281282322830895B5
:1045B00020912301222329F02091B30427FD0C949C
:1045C000AF220C94882220912301222329F02091EC
:1045D000B30427FD0C94C3220C94A2222091230142
:1045E000FC013296222331F08091B30487FF02C090
:1045F0008EE101C086E0DF011D928A95E9F70895FA
:1046000008950C9400230C940023CF930E9403235D
:104610000E946C0B0E940123C0E08C2F0E941A0B99
:10462000811104C0CF5FC530C1F701C081E0CF91D7
:1046300008950C9400230C9419230E941B2380914D
:10464000B904843049F11092670220E488E190E0D7
:104650000FB6F894A895809360000FBE2093600079
:1046600080E00E947B060E941B2383B7817F8460C9
:1046700083BF83B7816083BF7894889583B78E7F2B
:1046800083BF0FB6F894A8958091600088618093ED
:104690006000109260000FBE08950C9400230E94E9
:1046A000141B0E9477160E947B060C944D231F92C8
:1046B0000F920FB60F9211248F939F93AF93BF93D6
:1046C00080916702811113C08091AF049091B00472
:1046D000A091B104B091B2044196A11DB11D809387
:1046E000AF049093B004A093B104B093B204BF910F
:1046F000AF919F918F910F900FBE0F901F901895C3
:1047000082E084BD93E095BD9AEF97BD80936E00E3
:1047100008952FB7F8948091AF049091B004A091C0
:10472000B104B091B2042FBF0895CF92DF92EF92FF
:10473000FF920F931F932FB7F8944091AF045091BD
:10474000B0046091B1047091B2042FBF6A017B0183
:10475000EE24FF248C0120E030E0C016D106E206F2
:10476000F30610F4415051099A01281B390BC90175
:104770001F910F91FF90EF90DF90CF900895789464
:104780001F920F920FB60F9211248F939F93AF93A6
:10479000BF938091AF049091B004A091B104B09107
:1047A000B2040196A11DB11D8093AF049093B00493
:1047B000A093B104B093B204BF91AF919F918F9138
:1047C0000F900FBE0F901F90189581E08093E0002E
:1047D00080E28093D8001092C9008FE19EE4019797
:1047E000F1F700C0000087E090EBDC018093C20489
:1047F0009093C304A093C404B093C5049CE088E1E3
:104800000FB6F894A895809360000FBE9093600057
:10481000FFCF0E94F621811102C00E9470220E94E7
:104820000122809366020E94092290E09093B404D2
:104830008093B3040E940522682F70E080E090E02E
:104840000C94211F80918802089508950895CF93B4
:10485000DF93EC010E94FA25823011F08430D9F503
:1048600080912301882339F08091B30487FF03C02E
:1048700060E282E002C068E081E08093E9008FEFAF
:104880009091E800815095FD06C095ED9A95F1F75D
:1048900000008111F5CF8091E80085FF1CC0809158
:1048A0002301811105C040E050E068E070E003C0E2
:1048B00070E040E050E0CE010E9417268091E800B1
:1048C0008E778093E80080E2FE01A8E6B2E00190D6
:1048D0000D928A95E1F7DF91CF9108950895809127
:1048E000B804811109C00E94A8270E940528809160
:1048F000E20084608093E20008951092B804089565
:10490000089508950C944F2342E061EC81E00E94E9
:10491000212742E261EC82E00C9421278091BB04C4
:10492000833009F460C030F4813071F0823009F4D2
:1049300099C008958A3009F485C08B3009F46BC0A2
:10494000893009F0A7C020C08091BA04813A09F0EB
:10495000A1C08091E800877F8093E8008091BE0429
:104960009091BF04892B21F460E288E692E003C0B5
:1049700060E080E090E070E00E9462268091E800B4
:104980008B778093E80008958091BA04813209F012
:1049900081C08091BE049091BF04029708F07AC054
:1049A0008091E800877F8093E8008091E80082FD95
:1049B00005C08091B9048111F8CF6CC02091F3003B
:1049C0008091F20090E0922B029729F48091F100FF
:1049D0008B7F813021F48091F10080938802809157
:1049E000E8008B7753C08091BA04813A09F052C035
:1049F0008091BE049091BF04892B09F04BC0809137
:104A0000E800877F8093E8008091E80080FFFCCF7A
:104A10008091230136C08091BA048132D9F580910A
:104A2000BE049091BF04892BA9F58091E800877F8F
:104A30008093E8000E9456278091BC048093230154
:104A40000C94141B8091BA04813221F58091E80006
:104A5000877F8093E8000E9456278091BD04809351
:104A6000890208958091BA04813AA1F48091E80006
:104A7000877F8093E8008091E80080FFFCCF8091E1
:104A800089028093F1008091E8008E778093E8009E
:104A90000C945627089584B7877F84BF0FB6F89487
:104AA000A8958091600088618093600010926000FA
:104AB0000FBE80E880936100109261000E94D916B9
:104AC0000E94A8270E9405288091E20084608093BC
:104AD000E20078940E949A2A0E94E11689E191E00E
:104AE0000E9472168091B904853069F40E941D23DA
:104AF0008091B7048823B1F30E940523882391F3A2
:104B00000E940126EFCF0E94EE160E944411EACFC8
:104B10000C948A25292F332723303105C9F060F4FE
:104B20002130310581F02230310509F04AC08BE394
:104B300090E02DEC39E049C02132310511F12232EB
:104B4000310579F13EC082E190E028E03AE03DC0D5
:104B500099278130910561F040F08230910559F03C
:104B6000039779F5E3E9F9E008C0E9ECF9E005C05D
:104B7000E9EAF9E002C0E9E9F9E0849190E09F01F7
:104B800024C06115710541F061307105D1F489E0EF
:104B900090E028EF39E019C089E090E02FED39E08E
:104BA00014C06115710541F06130710551F48BE35A
:104BB00090E02AE13AE009C080E490E025E53AE09F
:104BC00004C080E090E020E030E0FA0131832083EF
:104BD00008950895CF93C82F0E94E925C0938A02B3
:104BE000CF9108958091B904843011F081E0089547
:104BF00082E0089580918A02811102C00C94F2250E
:104C0000089580E189BD82E189BD09B400FEFDCF30
:104C10008091D8008F7D8093D8008091E0008260E1
:104C20008093E0008091E00081FDFCCF0895CF9259
:104C3000DF92EF92FF920F931F93CF93DF93EC01DC
:104C40008B017A010E947527811133C0E114F104B0
:104C500039F0F70180819181081B190BC80FD91F0A
:104C6000C12CD12C0115110519F18091E80085FDA9
:104C700016C08091E8008E778093E800E114F1047B
:104C800049F0F70180819181C80ED91ED182C0827E
:104C900085E00FC00E947527882321F30AC08991FF
:104CA0008093F10001501109FFEFCF1ADF0ADACF2C
:104CB00080E0DF91CF911F910F91FF90EF90DF90F7
:104CC000CF9008952091C0043091C1042617370772
:104CD00048F06115710539F42091E8002E77209392
:104CE000E80001C0B901FC0120E06115710579F10E
:104CF0008091B9048823F1F18530F1F18091E800C9
:104D000083FD3CC08091E80082FD2EC08091E800C8
:104D100080FFEBCF2091F3008091F20090E0922B86
:104D20006115710551F08830910538F42191209377
:104D3000F100615071090196F3CF21E0089709F065
:104D400020E08091E8008E778093E800CECF21119B
:104D5000CFCF0AC08091B904882361F0853061F01B
:104D60008091E80083FD0AC08091E80082FFF2CFC5
:104D700080E0089582E0089583E0089581E0089539
:104D80002091C0043091C1042617370748F06115FF
:104D9000710539F42091E8002E772093E80001C0D6
:104DA000B901FC0120E06115710591F18091B90410
:104DB000882309F440C0853009F43FC08091E800A1
:104DC00083FD3DC08091E80082FD2FC08091E80006
:104DD00080FFE9CF2091F3008091F20090E0922BC8
:104DE0006115710559F08830910540F424912093A4
:104DF000F1003196615071090196F2CF21E00897D8
:104E000009F020E08091E8008E778093E800CBCF16
:104E10002111CCCF0AC08091B904882361F085307C
:104E200061F08091E80083FD0AC08091E80082FF74
:104E3000F2CF80E0089582E0089583E0089581E054
:104E40000895982F973068F59093E900981739F0F6
:104E50007091EC002091ED005091F00003C0242FE0
:104E6000762F50E021FD02C09F5FECCF3091EB0028
:104E70003E7F3093EB003091ED003D7F3093ED00AD
:104E80003091EB0031603093EB007093EC00209395
:104E9000ED005093F0002091EE0027FDE5CF80E07B
:104EA00008958F708093E90081E008958091BA049D
:104EB00087FF11C08091E80082FD05C08091B90490
:104EC0008111F8CF11C08091E8008B770BC08091E1
:104ED000B904882349F08091E80080FFF8CF8091E1
:104EE000E8008E778093E80008952091E4003091E7
:104EF000E50095E64091EC00842F817040FF23C0CF
:104F00008091E80080FD1DC08091B904882399F04C
:104F1000853099F08091EB0085FD11C04091E4004F
:104F20005091E5002417350729F3915011F09A01AB
:104F3000E1CF84E0089582E0089583E0089581E060
:104F4000089580E008954091E80042FFDDCF089584
:104F50000E9416280E941E28E0EEF0E08081816009
:104F60008083E8EDF0E080818F77808319BCA7ED26
:104F7000B0E08C918E7F8C9380818F7E80831092A5
:104F8000B80408950F931F93CF93DF930E941628C0
:104F90000E941E28C8EDD0E088818F7788838881A1
:104FA0008068888388818F7D888319BC1092B904BA
:104FB0001092B5041092B7041092B60400EE10E0FF
:104FC000F80180818B7F808388818160888342E0C3
:104FD00060E080E00E942127E1EEF0E080818E7F9A
:104FE0008083E2EEF0E08081816080838081886050
:104FF0008083F80180818E7F8083888180618883AF
:10500000DF91CF911F910F910895E8EDF0E080813D
:105010008F7E8083E7EDF0E080818160808384E093
:1050200082BF81E08093B8040C94C227E8EDF0E0E1
:1050300080818E7F80831092E20008951092DA00C2
:105040001092E10008951F920F920FB60F92112453
:105050002F933F934F935F936F937F938F939F9380
:10506000AF93BF93EF93FF938091E10082FF0BC05A
:105070008091E20082FF07C08091E1008B7F8093E6
:10508000E1000E94992A8091DA0080FF1FC0809180
:10509000D80080FF1BC08091DA008E7F8093DA00F9
:1050A0008091D90080FF0DC080E189BD82E189BD7A
:1050B00009B400FEFDCF81E08093B9040E946F2403
:1050C00005C019BC1092B9040E947D248091E100B2
:1050D00080FF19C08091E20080FF15C08091E2003E
:1050E0008E7F8093E2008091E20080618093E200F5
:1050F0008091D80080628093D80019BC85E08093AD
:10510000B9040E9481248091E10084FF30C0809125
:10511000E20084FF2CC080E189BD82E189BD09B431
:1051200000FEFDCF8091D8008F7D8093D8008091C4
:10513000E1008F7E8093E1008091E2008F7E80937A
:10514000E2008091E20081608093E2008091B504EA
:10515000882311F084E007C08091E30087FD02C03E
:1051600081E001C083E08093B9040E948224809191
:10517000E10083FF29C08091E20083FF25C0809178
:10518000E100877F8093E10082E08093B904109270
:10519000B5048091E1008E7F8093E1008091E20070
:1051A0008E7F8093E2008091E20080618093E20034
:1051B00042E060E080E00E9421278091F00088605A
:1051C0008093F0000E948024FF91EF91BF91AF91F6
:1051D0009F918F917F916F915F914F913F912F910F
:1051E0000F900FBE0F901F9018951F920F920FB641
:1051F0000F9211242F933F934F935F936F937F935D
:105200008F939F93AF93BF93CF93DF93EF93FF93CE
:10521000C091E900CF708091EC00D82FD17080FD53
:10522000D0E81092E9008091F000877F8093F00031
:1052300078940E9439291092E9008091F0008860EA
:105240008093F000CD2BCF70C093E900FF91EF91D8
:10525000DF91CF91BF91AF919F918F917F916F918E
:105260005F914F913F912F910F900FBE0F901F9024
:1052700018951F93CF93DF93CDB7DEB7AA970FB6DC
:10528000F894DEBF0FBECDBFEAEBF4E08091F100F1
:10529000819324E0E23CF207C9F70E948E248091BA
:1052A000E80083FF2EC18091BA049091BB04492F7E
:1052B00050E04A30510508F024C1FA01E556FF4F8D
:1052C0000C94E92A803821F0823809F01AC108C00C
:1052D0008091B6049091B704992389F082600FC041
:1052E0008091BE048F70873008F00BC18093E90075
:1052F0008091EB0085FB882780F91092E90090915E
:10530000E800977F9093E8008093F1001092F100FD
:10531000D1C0282F2D7F09F0F4C0882319F08230E6
:1053200061F0EFC08091BC04813009F0EAC0933095
:1053300009F080E08093B7042EC08091BC048111F5
:105340002AC08091BE048F702FEF280F263008F0FE
:10535000D8C08093E9002091EB0020FF1CC093305F
:1053600021F48091EB00806214C09091EB00906179
:105370009093EB0021E030E0A90102C0440F551FDB
:105380008A95E2F74093EA001092EA008091EB00E0
:1053900088608093EB001092E9008091E800877F9D
:1053A0008093E8000E945627ACC08111AAC01091DA
:1053B000BC041F778091E3008078812B8093E30009
:1053C0008091E800877F8093E8000E9456278091B3
:1053D000E80080FFFCCF8091E30080688093E300C9
:1053E000111102C082E001C083E08093B90489C03A
:1053F0008058823008F085C08091BC049091BD0433
:105400008C3D53E0950779F583E08A838AE28983AE
:105410004FB7F894DE01139620E03EE051E2E32F0F
:10542000F0E050935700E49120FF03C0E295EF7045
:105430003F5FEF708E2F90E0EA3010F0C79601C00A
:10544000C0968D939D932F5F243149F74FBF809174
:10545000E800877F8093E8006AE270E0CE01019661
:105460000E94622616C06091BE047091BF04AE0116
:105470004F5F5F4F0E948825BC01892B09F441C012
:105480009091E800977F9093E80089819A810E942B
:10549000C0268091E8008B778093E80032C0803886
:1054A00081F58091E800877F8093E8008091B504C2
:1054B0008093F1008091E8008E7772CF811121C036
:1054C0008091BC049091BD0499270297D4F48091F7
:1054D000E800877F8093E8008091BC048093B50446
:1054E0000E9456278091B504811106C08091E30087
:1054F00087FD02C081E001C084E08093B9040E946E
:1055000084248091E80083FF0AC08091E800877FAF
:105510008093E8008091EB0080628093EB00AA9674
:105520000FB6F894DEBF0FBECDBFDF91CF911F91B4
:1055300008950895CF938091B9048823A1F0C09174
:10554000E900CF709091EC00892F817090FD80E888
:10555000C82B1092E9008091E80083FD0E94392950
:10556000CF70C093E900CF910895991B79E004C0F2
:10557000991F961708F0961B881F7A95C9F7809592
:105580000895AA1BBB1B51E107C0AA1FBB1FA6178A
:10559000B70710F0A61BB70B881F991F5A95A9F7DC
:1055A00080959095BC01CD01089597FB072E16F4C8
:1055B000009407D077FD09D00E94C12A07FC05D0CE
:1055C0003EF4909581959F4F0895709561957F4F1A
:1055D0000895EE0FFF1F0590F491E02D0994FB0153
:1055E000DC0102C005900D9241505040D8F708955B
:1055F000FC014150504030F001900616D1F7319730
:10560000CF010895882799270895FB01DC0104C084
:105610008D910190801921F441505040C8F7881BAA
:10562000990B0895AEE0B0E0E8E1FBE20C94292E7E
:105630000D891E898F89988D26E02C831A83098312
:1056400097FF02C080E090E801979E838D83AE01B2
:10565000455E5F4F698D7A8DCE0101960E94422B87
:105660004D815E8157FD0AC02F813885421753074F
:105670000CF49A01F801E20FF31F10822E96E4E079
:105680000C94452EABE0B0E0E8E4FBE20C941B2E5A
:105690006C017B018A01FC0117821682838181FFE4
:1056A000CCC1CE0101963C01F6019381F70193FD37
:1056B000859193FF81917F01882309F4BAC18532D6
:1056C00039F493FD859193FF81917F01853229F40F
:1056D000B60190E00E94392DE7CF912C212C312C7E
:1056E000FFE1F315D8F08B3279F038F4803279F09D
:1056F0008332A1F4232D20611DC08D3261F08033EF
:1057000069F4232D216016C0832D8260382EE32D8D
:10571000E4603E2E2AC0F32DF8601DC037FC2DC07A
:1057200020ED280F2A3040F08E32B9F436FC81C1CA
:10573000232D2064322E19C036FE06C08AE0989EC2
:10574000200D1124922E11C0EAE02E9E200D11246E
:10575000222EF32DF0623F2E08C08C3621F4832DCB
:105760008068382E02C0883641F4F70193FD859198
:1057700093FF81917F018111B3CF982F9F7D955425
:10578000933028F40C5F1F4F9FE399830DC083363D
:1057900031F0833771F0833509F059C021C0F80129
:1057A000808189830E5F1F4F88248394912C53013D
:1057B00013C02801F2E04F0E511CF801A080B18007
:1057C00036FE03C0692D70E002C06FEF7FEFC501A8
:1057D0000E942E2D4C018201F32DFF773F2E16C023
:1057E000280122E0420E511CF801A080B18036FE53
:1057F00003C0692D70E002C06FEF7FEFC5010E940A
:10580000232D4C01F32DF0683F2E820133FC1BC089
:10581000822D90E088169906B0F4B60180E290E0FF
:105820000E94392D2A94F4CFF50137FC859137FE7B
:1058300081915F01B60190E00E94392D21102A94D8
:1058400021E0821A91088114910471F7E8C084362E
:1058500011F0893641F5F80137FE07C0608171818A
:10586000828193810C5F1F4F08C060817181072E78
:10587000000C880B990B0E5F1F4FF32DFF763F2E08
:1058800097FF09C090958095709561957F4F8F4FD8
:105890009F4FF0683F2E2AE030E0A3010E94752D53
:1058A000882E861845C0853731F4232D2F7EB22EE1
:1058B0002AE030E025C0932D997FB92E8F36C1F0B4
:1058C00018F4883579F0B5C0803719F0883721F0A1
:1058D000B0C0E92FE061BE2EB4FE0DC0FB2DF46018
:1058E000BF2E09C034FE0AC0292F2660B22E06C082
:1058F00028E030E005C020E130E002C020E132E0E5
:10590000F801B7FE07C060817181828193810C5FCD
:105910001F4F06C06081718180E090E00E5F1F4FD5
:10592000A3010E94752D882E8618FB2DFF773F2E30
:1059300036FE0DC0232D2E7FA22E891458F434FE7E
:105940000BC032FC09C0832D8E7EA82E05C0B82C5A
:10595000A32C03C0B82C01C0B92CA4FE0FC0FE01BB
:10596000E80DF11D8081803321F49A2D997EA92EB6
:1059700009C0A2FE06C0B394B39404C08A2D8678F1
:1059800009F0B394A3FC11C0A0FE06C0B21488F4C1
:10599000280C922C9B180EC0B21460F4B60180E261
:1059A00090E00E94392DB394F7CFB21418F42B185D
:1059B00002C0982C212CA4FE10C0B60180E390E018
:1059C0000E94392DA2FE17C0A1FC03C088E790E019
:1059D00002C088E590E0B6010CC08A2D867859F0A7
:1059E000A1FE02C08BE201C080E2A7FC8DE2B601FD
:1059F00090E00E94392D891438F4B60180E390E0DC
:105A00000E94392D9A94F7CF8A94F301E80DF11D85
:105A10008081B60190E00E94392D8110F5CF2220BF
:105A200009F442CEB60180E290E00E94392D2A941A
:105A3000F6CFF6018681978102C08FEF9FEF2B96FC
:105A4000E2E10C94372EFC0105906150704001108A
:105A5000D8F7809590958E0F9F1F0895FC01615097
:105A6000704001900110D8F7809590958E0F9F1F80
:105A700008950F931F93CF93DF93FB01238121FDA3
:105A800003C08FEF9FEF2CC022FF16C046815781C5
:105A9000248135814217530744F4A081B1819D01CF
:105AA0002F5F3F4F318320838C93268137812F5F77
:105AB0003F4F3783268314C08B01EC01FB01008428
:105AC000F185E02D0995892BE1F6D80116968D9187
:105AD0009C911797019617969C938E931697CE01DB
:105AE000DF91CF911F910F910895FA01AA272830D5
:105AF00051F1203181F1E8946F936E7F6E5F7F4F9B
:105B00008F4F9F4FAF4FB1E03ED0B4E03CD0670F16
:105B1000781F891F9A1FA11D680F791F8A1F911D69
:105B2000A11D6A0F711D811D911DA11D20D009F4B9
:105B300068943F912AE0269F11243019305D3193FB
:105B4000DEF6CF010895462F4770405D4193B3E0E4
:105B50000FD0C9F7F6CF462F4F70405D4A3318F08B
:105B6000495D31FD4052419302D0A9F7EACFB4E03C
:105B7000A6959795879577956795BA95C9F70097F4
:105B80006105710508959B01AC010A2E0694579595
:105B9000479537952795BA95C9F7620F731F841FEC
:105BA000951FA01D0895F999FECF92BD81BDF89A69
:105BB000992780B50895A6E1B0E044E050E00C9448
:105BC0000D2EA8E1B0E042E050E00C940D2E262FFF
:105BD000F999FECF92BD81BDF89A019700B40216E3
:105BE00039F01FBA20BD0FB6F894FA9AF99A0FBE91
:105BF00008950396272F0E94E82D0E94E72D252F58
:105C00000E94E82D242F0C94E82D0196272F0E9446
:105C1000E82D0C94E72DDC01CB01FC01F999FECFB6
:105C200006C0F2BDE1BDF89A319600B40D92415024
:105C30005040B8F708952F923F924F925F926F9223
:105C40007F928F929F92AF92BF92CF92DF92EF920C
:105C5000FF920F931F93CF93DF93CDB7DEB7CA1B8D
:105C6000DB0B0FB6F894DEBF0FBECDBF09942A88B8
:105C7000398848885F846E847D848C849B84AA8460
:105C8000B984C884DF80EE80FD800C811B81AA81ED
:105C9000B981CE0FD11D0FB6F894DEBF0FBECDBFB8
:085CA000ED010895F894FFCF17
:105CA800010209090901191A1B1C1D1E1F202122A6
:105CB8000021007F22000343022224272425246E8A
:105CC800242624015247423A25634D3A202532645E
:105CD8000A683A20253264733A20253264763A20DD
:105CE8002532640A00313332366697C634350001EE
:105CF800020202020606060909090909090F0F0F1F
:105D08000F0F0F1515151819191919191919191926
:0C5D1800192324000810181810080000BF
:00000001FF
